:03000000021D607E
:0C1D600078FFE4F6D8FD7581E102003642
:0100190022C4
:061A52008B2C8A2D892E69
:101A5800751A027F48121BD6121DB1EF20E0F9ABB0
:101A68002CAA2DA92E1209F97873E6FE08E6FDEDD9
:011A7800FF6E
:011A7900224A
:100FCC00434647002D53322D0052415445434C5259
:100FDC0020554E49544C4954455452494754524556
:100FEC00565354525453544F505A45524F424155F4
:100FFC004444464C5453415645525354205043207C
:10100C00205F3120735F3220735F35207331207382
:10101C002032207320352073203130207333302060
:10102C007331206D2032206D2035206D2031302021
:10103C006D3330206D31206820000000010002006B
:10104C0005000A001400320064012C025804B00B95
:10105C00B8177046508CA001020408103046656524
:10106C0074596172644D6574724F6666204F6E20C0
:10107C00204E6F2020596573204F66662054696D91
:10108C0065416C7420547269674F666620547269AE
:09109C00675374727452656320FD
:101B360025E02445F582E43410F58322052EE52EB2
:101B4600C3940222A62EE52E75F004A42208F608F8
:041B5600F608F62275
:10177800789376AB0876CD08760008760AE408F602
:1017880008760108F6087664087640121B5308F6B6
:1017980078A1F608760A08F608763C08F608761462
:0F17A80008F608760F121B5378AE7605021B1257
:10197700751E1D751FC01216307894E664CD70046D
:1019870018E664AB600312177878ADE6FFF46003DE
:0F199700EF700478AD760178AEE6B4FF02760506
:0119A600221E
:0D1D3600C2AF7DC07C1DE4FF121C7CD2AF4B
:011D4300227D
:101630007539FF851E3A851F3B753C00753D007569
:101640003E93E4FFAB39AA3AA93B8F82758300121F
:1016500009CCAB3CAA3DA93E8F82758300120A0BD0
:101660000FBF1CE078ACE6FFF46003EF700478ACC9
:02167000760101
:011672002255
:101B12007D01E4FF121B9B121D36C2AF7F937B1C1B
:101B22007DC07C1D121C86D2AF7F021218A5E4FD77
:041B3200FF021B9BF8
:10050E00E4F52C7BFF7A0F79CC1217387F05121881
:10051E00A5A297829650FAA2969219A297921AE5E0
:10052E002C75F004A424D5F9740F35F0FA7BFF1264
:10053E0017387F051218A5852C2DE4F52E7BFF7A32
:10054E000F79D0121738E52CB40A0040030205DCEF
:10055E00900565F82828730205830205DC0205A4C0
:10056E000205AC0205B00205B80205C00205C402C0
:10057E0005CC0205D47F01EF121B367895E6FC08F8
:10058E00E6FD7401936D7003E4936C70028F2E0F71
:10059E00BF0FE40206627897E6F52E02068578987C
:1005AE00800278A0E6F52E02069F789FE6F52E02D1
:1005BE0006CD78A9800278AAE6F52E0206EA78AB77
:1005CE00E6F52E02071F78AEE6F52E020745E52C5E
:1005DE00652D600302052DA219309601B35013A2AA
:1005EE0096921930960C052CE52CC3940D4003E41D
:1005FE00F52CA21A309701B350D4A297921A3097C5
:10060E00CDE52CB40D0050C690061DF828287302B7
:10061E00064402066D0206730206910206AB02063E
:10062E00BF0206D80206F502070D0207330207566F
:10063E0002075C020762052EE52EC3940F40037578
:10064E002E01E52E121B36E493FF7401937895CF9D
:10065E00F608EFF6121B4C2409F974100207281243
:10066E00145C0205DC052EE52EC394034003E4F56D
:10067E002E7897A62EE52E75F004A42469F9741031
:10068E00020728121B424003E4F52E7898A62EE5A9
:10069E002E75F004A42475F97410020728121B425B
:1006AE004003E4F52E78A0121B4A2475F9741080CD
:1006BE0069121B424003E4F52E789FA62EE52E7597
:1006CE00F004A4247DF974108050052EE52EC394F9
:1006DE00044003E4F52E78A9A62EE52E75F004A4A9
:1006EE002485F974108033052EE52EC39403400340
:1006FE00E4F52E78AA121B4A2485F97410801B0586
:10070E002EE52EC394044003E4F52E78ABA62EE519
:10071E002E75F004A42495F9741035F0FA7BFF12AF
:10072E0017380205DC052EE52EC394064003E4F5CA
:10073E002E78AEA62EE52E9010639375F018A4FFBA
:10074E00AEF012128A0205DC1217780205DC121BBB
:0A075E00120205DC43A2080205DCCC
:0A1D84004552415300444F4E450004
:101D06007895E6F54F08E6F55022E564AE63780669
:011D160022AA
:1011FE00C217C21878ADE6FFE4FCFDFEFB7A20F9BB
:10120E00F8120A2D8F6A8E698D688C67E47B40FA1E
:10121E00F9F8120AB88E618F62E4F52DF52EC3E54A
:10122E002E9562E52D9561501CE52C64816016AFFC
:10123E002EAE2D1219A7121C688F2C052EE52E70BE
:10124E00DD052D80D9E52CB48108E52E152E700212
:10125E00152DE52E65627004E52D6561700CD217B3
:10126E00121D44E4F563F5648007852D63852E64B5
:0B127E00E4F565F566754E80121D0654
:011289002242
:1019A700C3EF9562EE95615024EF7806C333CE33CB
:1019B700CED8F9FD751A02EE7873F6CFEDCFEF08A2
:0D19C700F67F50121C26121DB1EF20E0F932
:0119D40022F0
:031C0C00CDEFCD4C
:101C0F00751A02EE7873F6ED08F67F50121C261245
:061C1F001DB1EF20E0F909
:011C2500229C
:101C6800751A017F50121BD6121DB1EF20E0F978CA
:031C780073E6FF11
:011C7B002246
:101C5300121C0CE4FFFE0FBF00010EBE0FF8BFA065
:041C6300F5121C68F2
:011C6700225A
:0618DB00CBEFCBCAEECA00
:1018E100301703301827751A03EA7873F6EB08F6F8
:1018F10008EDF67F50121C26121DB1EF20E0F9E42D
:0D190100FFFE0FBF00010EBE0FF8BFA0F5E6
:01190E0022B6
:1016B600752F0075300075314EE4F52E121D10C3DE
:1016C60033CE33CED8F97C00252EFFEC3EFEAB2F71
:1016D600AA30A931852E827583001209CCFD121815
:1016E600DB052EE52EC3940640D2756500756606A9
:0116F60022D1
:10138B008E2C8F2D121D10C333CE33CED8F925667C
:10139B00FFE5653EFEEEC0E0EFC0E0E52CFDD0E0E2
:1013AB00FFD0E0FE1218DB0566E5667002056512DC
:1013BB001D10C333CE33CED8F92566FFE5653EFE4F
:1013CB00AD2D1218DB0566E566700205650552E565
:1013DB005270020551C3E5669440E56594004017D1
:1013EB00E4F565F5660564E564700205639562E5F1
:0813FB006395614002D2172244
:10145C00E4F565F5667BFF7A1D7984121738D2188E
:10146C00E4F539F53AC3E53A9562E53995615021D1
:10147C00E53AAE397806C333CE33CED8F9F5668E5D
:10148C00657D81FF1218DB053AE53A70D805398085
:10149C00D4C2187BFF7A1D7989121738E4F563F5ED
:0714AC0064F565F566C21747
:0114B3002216
:10140300E4F539F53AF53BF53CC3E53C9562E53B3C
:1014130095615044E53A6481603EAF3CAE3B12199E
:10142300A7121C688F3AE53A64807022AF390539F8
:10143300FCFDFEFBFAF9120DA37F2C120016AE3B46
:10144300AF3CE4FCFDFBFAF9120DA3121DA1053C10
:08145300E53C70B5053B80B1DA
:01145B00226E
:0215A5008F397C
:1015A700E4F53AF53BF53CF53DC3E53D9562E53C91
:1015B70095615030E53B6481602AAF3DAE3C12191E
:1015C700A7121C688F3BE53BB4800FE53A6539707D
:1015D70007AF3DAE3C0219A7053A053DE53D70C989
:0415E700053C80C57A
:0115EB0022DD
:1016F700121D0678A0E6F553E4F551F5521216B619
:1017070085636B85646C7F01121AA130021A78A376
:10171700E6FE08E6FFE4FCFD7B64FAF9F8120A2D01
:101727008F608E5F8D5E8C5D300505C205121C3D96
:01173700228F
:1018310085632C85642DE56645656008052DE52DDC
:101841007002052C856B63856C641216B6852C635A
:10185100852D64C3E52D9562E52C95614007E4F57E
:0A18610063F564D2177F02021AA19A
:101C7C00740478FF769612FF0322740078FF769630
:041C8C0012FF03221E
:030033000210A513
:0D10A500C0E0C0F0C083C082C0D075D0088C
:1010B200E5D954F8FF120BD110DF0810DF1010EE43
:1010C2001811092010F028110930110B38111140A4
:1010D200110948112A5011475800001155851DDA8F
:1010E200C2DDC2DC751B00751C008070800EE51A23
:1010F20070028056051CE51C7002051B1200268F2B
:10110200DAC2DDC2DC80558016D2DDC2DC804DC27F
:10111200DDC2DCE51A7004C2DA8041D2DA803DC257
:10112200DDD2DC7518048034AFDA121D6C051CE5C3
:101132001C7002051BC2DDC2DCE51A7004C2DA8033
:101142001BD2DA8017AFDA121D6CC2DDD2DC751841
:0E115200028009751804C2DDC2DCD2DAC2DBED
:0B116000D0D0D082D083D0F0D0E0329D
:101A000043910C43920CE4F5DBEF25E0F5DB301954
:101A10000343DB0175DD1775DC1775D84453F8FEF9
:091A200053F7FEE4F518D2E822A8
:101C2600E51830E002FF22E4F519751803EF25E008
:071C3600F51DD2DD7F022243
:101BD600E51830E002FF22E4F519151A751805EF2D
:0B1BE60025E04401F51DD2DD7F022246
:061DB10020DBFDAF18224B
:0D002600151AAF19051974732FF8E6FF22A3
:0C1D6C0074732519F8EFF60519151A22FA
:0C1D7800E4F5847585FF53913FF592223D
:1019D500811902006F035D5733767E437F771004CC
:1019E500007B3E6C1F7C78773B020F382C5A1A6FB0
:0B19F500797518763C0E2F4E2B375DE5
:10186B004EFECCEFCC0F74732CF8EEF6EDC4332296
:10187B009019E5E493FF78D9F608EFF608F608F629
:10188B0022E493FF74D92EF8EFF60E22EE3395E097
:0A189B00FDFC227B007A0079D422C4
:10116B00E4FF0F2473F876CD0F74732401F87680A7
:10117B000F74732402F876E00F74732403F876F877
:10118B00301B0A0F74732404F87671800ACEEFCEED
:10119B000F74732EF8767078D9E6FEC4540FFDCC1D
:1011AB00EFCC0F74732CF8EDF6EEC454F0FE78DA36
:1011BB00E6FD131313541F12186B54E0FE78DBE695
:1011CB00FD1313543F12186B3354C0FE78DCE6FD4D
:1011DB00C31312186B33335480FECDEFCD0F7473E2
:1011EB002DF8EEF68F1A7F38121C26121DB1EF2048
:0211FB00E0F919
:0111FD0022CF
:10190F00C21B12187B751A0A787376CD0876800879
:10191F0076E00876F80876700876050876D50876AA
:10192F009B0876FFE408F67F38121C26121DB1EFD4
:03193F0020E0F9AC
:011942002282
:101BF100EF24F9600B14600C2402700EC21B8007E5
:0B1C0100D21B800312187B12116B2213
:1014B400C3EF648094E1400ED3EF648094FA500645
:1014C400EF24ACFF803CC3EF648094C1400ED3EFA3
:1014D400648094DA5006EF24CCFF8026C3EF648046
:1014E40094B0400ED3EF648094B9500674D02FFFAB
:1014F4008010BF2D047F0A8009BF5F047F0B800228
:031504007F0C2237
:101A7A00CEEDCECDEFCDCFEECF1214B4EF3395E04D
:101A8A00FE74D92FF58274193EF583E493FF74D955
:071A9A002DF8EFF602116BBD
:061738008B3B8A3C893D59
:10173E00E4FE9019E512188CBE04F7E4FEAB3BAA4A
:10174E003CA93D8E827583001209CCFF60191214DC
:10175E00B4EFFD3395E0FC74D92DF58274193CF588
:0A176E008312188CBE04D602116B22
:04128A008F828E833E
:10128E001218977B197AFC79FF78FFD3120B58400E
:10129E000390FC19AF82AE83121897E47B0F7A2766
:1012AE00F9F8C3120B58500390270FE4F52F74D49E
:1012BE00252FF8E4F6052FE52FB405F2AE83AF82A5
:1012CE0012189712189E120DA378D7E6701A752F62
:1012DE000374D3252FF8E6FF74D4252FF8EFF6D537
:1012EE002FEF78D4762080E112189E12173830082E
:1012FE000F7BFF7A1979D5121CF312189E121CF36C
:01130E0022BC
:101CE000C214C216C213E4FDFF121B9BE4FD7F0168
:031CF000021B9B39
:101B9B00EF146011047016BD0104C2828002D28260
:0E1BAB00A282921522BD0103C28122D28122A4
:101AA100EF24FE600D14601124027019D214756EBA
:101AB1000122C214A215928222D216756F027D01F3
:061AC1007F01121B9B22B5
:101A2900301412D56E0F308207C282756E0F800591
:101A3900D282756E23E56FD39400400CD56F09C22D
:091A490016E4FD7F01121B9B2233
:101C900046554C4C005A4C4F470020332D340054CD
:041CA00072696700FE
:101AED0078DEE6FE08E6FF22E6FE08E6FFE4FCFDF2
:101AFD002278CA120B9378C2020BACC3E55C94B882
:051B0D00E55B940B22D2
:03001300021B5A73
:101B5A00C0E0C0D075D010200F0CAF8DEFAD8BF563
:101B6A0058EDF559D20F758D00758B00D0D0D0E0A5
:011B7A003238
:0218A5008F3A78
:1018A700E4F53BF53CC3E53C953AE53B9400502312
:1018B700900000AF82AE83E4FCFD7B207A4EF9F8FE
:1018C700D3120B584003A380EA053CE53C70D605CC
:0318D7003B80D281
:0118DA0022EB
:0E1D44007BFF7A1C79901217387F0A0218A5CF
:0F1D2700D20D301706121D44C20D221216F722DC
:05000E00C20D021831D3
:101C3D0078CE120BB800000000121AFE78CA120BF3
:061C4D00B80000000022B7
:101D17008E2C8F2DEEFF120016AF2DE52D0200162B
:10003600121D78121D8E121CE07F041218A520973F
:100046000B7D057F0112130FD2AF80FE209612D2D0
:10005600AF121977C2197F70121A001211FE12051B
:100066000E121977120504D2AFC2197F70121A0048
:100076007F011218A51211FE12190F7A1C7995121A
:1000860004F97A1C799A1204F9120019E4F572122D
:1000960017F67F011218A5E478D2F608F612001AB0
:1000A600A2969209A297920AE4F52478C6120BB892
:1000B60000000000E4F52578CE120BB8FFFFD8F15A
:1000C60078C2120BB800000000C20B78CA120BB837
:1000D60000000000C20EC212C20DE4F526F527C2CA
:1000E60008F55BF55CF558F559C20FF55AC210F5DF
:1000F60057F556F555F554F560F55FF55EF55DF582
:10010600207898E66004D2808002C28078A9E6242E
:10011600FE600B14600C2402700AD2018006D2061F
:100126008002D20078AAE624FE6007047006D20296
:100136008002D20778ABE624FE600B14600C240222
:10014600700AD2038006D2048002D205300117C29B
:100156000178A1121AF57B64FAF9F8120A2D8F5765
:100166008E568D558C54E572C3940240F9E4F572AF
:10017600A208B39281209605209702D211309635B7
:1001860030973230112FC21178C2120B93EC4D4EBC
:100196004F78CE700C120BB800000000121AFE80C9
:1001A60010120BB80000000078C2120BB800000055
:1001B60000D20AD209A209309601B3502AA2969219
:1001C6000930961C201119121B085014C201300B5D
:1001D60006C20B7F068004D20B7F07121BF1805BE1
:1001E600E4F55BF55C8054209651740A255CF55C59
:1001F600E4355BF55B121B084041E55C9410E55B5A
:1002060094275037755B27755C10300807C20812B3
:1002160005048027D2087D01E4FF12130F7F89129F
:1002260000167F011218A57F821200167F01121890
:10023600A57F841200167F31120016A20A3097019C
:10024600B35017A297920A30971020110DB20D30B5
:100256000D05121D27800312000E120768AF57AE58
:1002660056AD55AC54EC4D4E4F602674FF2FF557E6
:10027600EE34FFF556ED34FFF555EC34FFF554AF8B
:1002860057AE56AD55FC4D4E4F7006200D03121D50
:1002960027AF60AE5FAD5EAC5DEC4D4E4F60237434
:1002A600FF2FF560EE34FFF55FED34FFF55EEC34BD
:1002B600FFF55DAF60AE5FAD5EFC4D4E4F70031255
:1002C600000E200F03020370C2AFC20FD2AFE48547
:1002D600592B85582AF529F528AF2BAE2AAD29AC1E
:1002E600287B107A27F9F8120A2D8F2B8E2A8D2952
:1002F6008C28E4FB7A90F9F81215EC8F2B8E2A8D58
:10030600298C28789FE66009C374B89FFF740B9EFA
:10031600FEE55A14601624FE602024037049C3EFDC
:1003260094B0EE9404500E755A018009D3EF9414DC
:10033600EE94054035755A038030C3EF94B0EE94C1
:10034600045027755A01300006200D03121D273070
:100356000305C203121C3D300D02D2107BFF7A1C2E
:10036600799F1217388003E4F55A0525E525C394CD
:100376000150030204F3E4F525FB7A0079DD121A35
:100386005278DEEEF608EFF678DDE66402600302E8
:1003960004F378C6120B9FE8C0E0E9C0E0EAC0E0CB
:1003A600EBC0E0121AED7897E6FD121559D0E0FB86
:1003B600D0E0FAD0E0F9D0E0F8EB2FFFEA3EFEE914
:1003C6003DFDE83CFC78C6120BAC0524E524C3943D
:1003D6000550030204F378C6120B93E47B05FAF981
:1003E600F81215EC78C6120BAC78C6120B9378C2CD
:1003F600120B9FC3EF9BFFEE9AFEED99FDEC98FC66
:1004060078C6120BAC78CE120B9378C6120B9FD31C
:10041600120B58400A78C6120B9378CE120BAC30EA
:100426000B0C78CE120B9378E0EEF608EFF678C652
:10043600120B9378DEEEF608EFF6300B0308800217
:1004460078DEE6FE08E6FF12128A301206121AED70
:10045600121D170527E52770020526C3789696E52F
:100466002618964038E4F526F527300E06121AEDC2
:10047600121D17300D277F03121AA120171978A015
:10048600E6600C3010097F007E8212138BC21012B8
:100496001AED12138B8006121D4412000E78C61236
:1004A6000B9378CA120BAC78C6120BB8000000008A
:1004B600E4F524300405C204121C3D30061678A566
:1004C600121AF578CA120B9FD3120B584006200D4C
:1004D60003121D2730071678A7121AF578CA120BD1
:1004E6009FC3120B585006300D0312000E121A2924
:0304F60002016C94
:1004F9007BFF1217387F041218A52278AEE6FDE4B7
:05050900FF12130F2298
:101AC700444C0021536967005A4C4F47004D4F441F
:101AD70000332D34004E6F762032312032303036CD
:061AE7000050524F4700C1
:10167300AF34AE33AD32AC31EC4D4E4F22EF24FFDD
:10168300F534EE34FFF533ED34FFF532EC34FFF58A
:101693003122E475342075334EF532F53122E47589
:1016A3003401F533F532F53122752E00752F0075AF
:0316B3003093224F
:10076800121D52EF7003020993121BB9EF120BD13D
:10077800095A2409652A097E48096A5008B45207AB
:10078800A66108366309886808896C088F72088C26
:100798007308B874092A7609257800000993C20BF2
:1007A8007BFF7A1A79C7121738121695121D52EF65
:1007B800700A121673600512168080F01216737094
:1007C80003020993121BB98F2D1215A5E4F53412F3
:1007D80016A5E47F06FEFDFCAB34AA33A932A83186
:1007E800C3120B6E501F121C688F2D120016E534B1
:1007F8002401F534E43533F533E43532F532E435A4
:1008080031F53180CD121C688F2DE52D648060167E
:10081800E52D64816010120016121C688F2D1200DD
:1008280016752C018003E4F52CE52C70D8221216DD
:10083800AC1216A1F52D1216736024121695121D0E
:1008480052EF700A121673600512168080F01216A5
:10085800736003120994052DE52DC3941C40D7122B
:100868001673601A7893B6AB0708B6CD030209620F
:100878007BFF7A1A79CA1217387F0A0218A502096B
:1008880022B20E220214031216ACE4F52DAB2E058B
:1008980030E530AA2F7002052F14F91209B3FF12A0
:1008A8000016052DE52DC3941C40E22243A2082220
:1008B800C20B752E00752F007530701216A1F52D1C
:1008C8001216736024121695121D52EF700A121632
:1008D80073600512168080F0121673600312099473
:1008E800052DE52DC3940240D7121673602CAE7007
:1008F800AF71EE3395E0FDFC78CA120B9FC3EF9BF6
:10090800F538EE9AF537ED99F536EC98F535AF38B8
:10091800789DE537F608EFF68040021630C20B02E4
:10092800145C7A1A79CF1209A87A1A79D4121CF3AE
:1009380078ACE62430FF120016121DA17F76120053
:10094800167A1A79D81209A87A1A79DC121CF302D5
:100958001DA1C20BE4789DF608F6021B12C20B0219
:100968001778C20B7BFF7A1A79E81217387D017F56
:100978000112130F80FE7D03E4FF12130FD212221F
:0B09880078AEE6FDE4FF12130FC21270
:1009930022121BB9AB2EAA2FA930852D8275830095
:1009A300EF120A0B227BFF121CF3121DA17BFF2205
:0A1D8E00E4F5955396BF53A27F229F
:1017F6005389F0438901538FFE758C70E4F58A5343
:10180600B8FD53B7FDD2A9D28C53890F43899053A3
:101816008FEFF58DF58B4391105392EF53B8F75335
:0B182600B7F7D2ABD28ED28AD2AA2232
:03000B00021D983B
:091D98000572758C70758A003229
:03001B00021DAA19
:071DAA00758D00758B0032FE
:101CA4000D0A003031323334353637383941424346
:041CB400444546005D
:101CB800AF4DAB41AA42A943054D22AF40AE3FAD5F
:041CC8003EAC3D22CF
:10130F005387BF75985053877FE4F5BABF010543E4
:10131F00A240800353A2BFE4F5BDED146015146025
:10132F001A14601F1460242404702575BEF075BF55
:10133F000B802375BEF075BF05801B75BEF075BFA2
:10134F0002801375BE7075BF01800B75BEB0800330
:10135F0075BE30E4F5BF75BD035391FE4392014353
:10136F0091025392FDC21C53B8EF53B7EF43B8101D
:0C137F00E478C0F618F678C1F6D2AC2273
:030023000219437C
:10194300C0E0C0D075D01030981E78C0E6C3940FA5
:10195300501418E60624AFF8A69978C00618E6C313
:10196300941040027600C298309904C299C21CD0E8
:04197300D0D0E032BE
:08000300201CFDD21C8F992284
:101B7B0078C0E6D39400401508E60624AFF8E6FFDC
:0F1B8B0078C01608E6C394104005E4F6227F00E8
:011B9A002228
:03001600020003E2
:101BB9007F207E4E78C0E67010D3EF9400EE94003B
:0C1BC9004007EF1F70EE1E80EB121B7B2C
:011BD50022ED
:101CF3001209B3FF600C120016740129F9E43AFAD1
:031D030080EE224D
:0E1D520078C0E6D3940040037F01227F002278
:091DA1007BFF7A1C79A4021CF3FB
:0E0DA3008F408E3F8D3E8C3D8B418A428943AE
:100DB100E4F54DEC4D4E4F7017E94A4B70057F300D
:100DC100020016121CB88F827583007430020EC6A1
:100DD100121CC5EC33502AE5434542454170077F5B
:100DE1002D120016800D121CB88F82758300742D90
:100DF100120A0B121CC3120B4A8F408E3F8D3E8C80
:100E01003D754C017547007546CA75459A75443B59
:100E1100E4FFFEFDFCAB47AA46A945A844D3120B4B
:100E21006E5003020EB1121CC3A844120AB88F4BB4
:100E31008E4A8D498C48EC4D4E4F7004E54C702321
:100E4100E54B2430FFE5434542454170051200164C
:100E5100800EAE4D121CBA8E82758300EF120A0B02
:100E6100E4F54CAF47AE46AD45AC44AB4BAA4AA9FD
:100E710049A848120A2DCAEECAC9EDC9C8ECC8C3AF
:100E8100E5409FF540E53F9AF53FE53E99F53EE5A2
:100E91003D98F53DAF47AE46AD45AC44E47B0AFA1B
:100EA100F9F8120AB88F478E468D458C44020E110F
:100EB100E542454345416010AB41AA42A943854DF6
:080EC10082758300E4120A0BA4
:010EC9002206
:100BF7000134C35001DBBF68028BBB800344B79845
:100C07000407B3B004D5AFC805A9ABE00689A7F8B8
:100C17000775A410086DA02809719C400A8198588F
:100C27000B9F94700CCA90880DE98CF90E048CA068
:100C37000EA88AAC0F4D88B80FF786C410A184D0D0
:100C4700115182DC120580E812BB7EF413747D001B
:100C570014307B0C14F2791815B877241680753088
:100C6700174B733C1819714818ED6F5419C46D6010
:100C77001AA16B6C1B7E69781C6167841D4A65909D
:100C87001E37639C1F2561A8201A5FB421125DC01F
:100C9700220D5BCC230E59D8241557E4251F55F098
:100CA700262F53FC27425208285B501429764E20E2
:100CB7002A9B4C2C2BC04A382CEE48442E1E4650FB
:100CC7002F55445C308F426831D1407433173E80D2
:100CD70034633C8C35B13A98370938A4386636B056
:100CE70039C734BC3B2D32C83C9D30D43E0F2EE073
:100CF7003F882CEC41062AF8428D29044418271016
:100D070045AB251C4741232848E121344A861F402B
:100D17004C311D4C4DE21B584F9C1964515D1770A7
:100D27005323157C54EF138856C4119458A20FA06F
:100D37005A830DAC5C6D0BB85E6009C4605807D070
:100D4700625A05DC646203E8667301F4688A00008E
:100D57006AA1FE0C6CB8FC186ECFFA2470E6F83066
:100D6700000000000000000000000000000000007C
:100D7700000000000000000000000000000000006C
:100D8700000000000000000000000000000000005C
:0C0D970000000000000000000000000050
:1017B70075F004E533A424F7F582E5F0340BF583DF
:1017C700E49322FE740193FF75F004E533A422F538
:1017D70083C37401939FFFE4939EFEE4228F348EAC
:0F17E700338D328C31228F308E2F8D2E8C2D2210
:101CCC00C3EF9DEE9C400AD3EF9BEE9A50037F012D
:041CDC00227F002241
:040ECA008E318F32A4
:100ECE00E4F5331217B7FC740193FD1217CF24FB10
:100EDE00F582E5F0340BF583E493FA740193FBAFDE
:100EEE0032AE31121CCCEF7003020FBA1217B712CA
:100EFE0017CA24FBF582E5F0340B1217D68F378E06
:100F0E0036F535F5341217CF24FDF582E5F0340BA6
:100F1E00F583E4931217CA24F9F582E5F0340B1227
:100F2E0017D68F3B8E3AF539F538AD39AC38120BF2
:100F3E004A8F3B8E3A8D398C38AE31AF32E4FCFDA0
:100F4E00EEC0E0EFC0E01217B7FE740193FBCAEEDD
:100F5E00CAD0E0FFD0E0FEC3EF9BFFEE9AFEED9409
:100F6E0000FDEC9400FCAB3BAA3AA939A838120A52
:100F7E002DAB37AA36A935A8341215ECC8ECC8C962
:100F8E00EDC9CAEECACBEFCB1217CF24F9F582E525
:100F9E00F0340BF583E493FE740193FFE4FCFDEB58
:100FAE002FFFEA3EFEED39FDEC38FC220533E5332A
:0D0FBE00C3946A5003020ED1E4FFFEFDFC57
:010FCB002203
:01001A0022C3
:101507001217E4AB34AA33A932A831E8C0E0789BBC
:10151700E6FE08E6FFE4FCFDD0E0F8120A2D1217FC
:10152700E4780E120B7F1217E4789DE6FE08E6FFBB
:10153700EE3395E0FDFCE5342FF534E5333EF53326
:10154700E5323DF532E5313CF531AF34AE33AD32FE
:02155700FC2274
:021559008D2CD7
:10155B00120ECA1217ED1215071217EDE52C1460B7
:10156B001C14702DE47FE87E03FDFCAB30AA2FA981
:10157B002EA82D120A2DE47BE87A0B800CAF30AE2F
:10158B002FAD2EAC2DE47B03FAF9F81215EC1217E4
:09159B00EDAF30AE2FAD2EAC2DEA
:0115A4002224
:1009B300BB010689828A83E0225002E722BBFE0242
:0909C300E32289828A83E4932275
:1009CC00BB010CE58229F582E5833AF583E02250E0
:1009DC0006E92582F8E622BBFE06E92582F8E2222A
:0D09EC00E58229F582E5833AF583E4932244
:1009F900BB010689828A83F0225002F722BBFE01DD
:020A0900F322D6
:100A0B00F8BB010DE58229F582E5833AF583E8F021
:100A1B00225006E92582C8F622BBFE05E92582C8CD
:020A2B00F222B5
:100A2D00E88FF0A4CC8BF0A42CFCE98EF0A42CFC68
:100A3D008AF0EDA42CFCEA8EF0A4CDA8F08BF0A4E6
:100A4D002DCC3825F0FDE98FF0A42CCD35F0FCEB45
:100A5D008EF0A4FEA9F0EB8FF0A4CFC5F02ECD390A
:0F0A6D00FEE43CFCEAA42DCE35F0FDE43CFC2277
:100A7C0075F008758200EF2FFFEE33FECD33CDCC31
:100A8C0033CCC58233C5829BED9AEC99E5829840B4
:100A9C000CF582EE9BFEED9AFDEC99FC0FD5F0D691
:100AAC00E4CEFBE4CDFAE4CCF9A88222B800C1B9BB
:100ABC000059BA002DEC8BF084CFCECDFCE5F0CBF9
:100ACC00F97818EF2FFFEE33FEED33FDEC33FCEB32
:100ADC0033FB10D703994004EB99FB0FD8E5E4F9ED
:100AEC00FA227818EF2FFFEE33FEED33FDEC33FCDA
:100AFC00C933C910D7059BE99A4007EC9BFCE99ACE
:100B0C00F90FD8E0E4C9FAE4CCFB2275F010EF2F12
:100B1C00FFEE33FEED33FDCC33CCC833C810D70712
:100B2C009BEC9AE899400AED9BFDEC9AFCE899F84D
:0E0B3C000FD5F0DAE4CDFBE4CCFAE4C8F922E0
:1015EC00C2D5E830E70FB2D5E4C39BFBE49AFAE42A
:1015FC0099F9E498F8EC30E717B2D5121622120AD2
:10160C00B8E4C39BFBE49AFAE499F9E498F88003F4
:10161C00120AB830D50DE4C39FFFE49EFEE49DFD95
:04162C00E49CFC221C
:0E0B4A00C3E49FFFE49EFEE49DFDE49CFC22BC
:100B5800EB9FF5F0EA9E42F0E99D42F0EC6480C814
:060B680064809845F022B4
:100B6E00EB9FF5F0EA9E42F0E99D42F0E89C45F0DD
:010B7E002254
:100B7F00E86010ECA2E713FCED13FDEE13FEEF138C
:040B8F00FFD8F02279
:0C0B9300E6FC08E6FD08E6FE08E6FF228E
:0D0B9F00E6FB08E6F908E6FA08E6CBF822C6
:0C0BAC00ECF608EDF608EEF608EFF62275
:100BB800D083D082E493F608740193F60874029304
:090BC800F608740393F67404733B
:100BD100D083D082F8E4937012740193700DA3A3B3
:100BE10093F8740193F5828883E4737402936860C7
:060BF100EFA3A3A380DFC7
:00000001FF
